:100000000C945B000C947E030C94AB030C94830063
:100010000C9483000C9483000C9483000C94830054
:100020000C9483000C9483000C9483000C94830044
:100030000C9483000C9483000C9483000C94830034
:100040000C94D8030C9483000C9494050C948300B6
:100050000C9483000C9483000C9483000C94830014
:100060000C9483000C948300000024272A000025B0
:10007000282B000023262904040404040404040299
:100080000202020202030303030303010204081035
:100090002040800102040810200102040810200002
:1000A0000000070002010000030406000000000039
:1000B00000000000940211241FBECFEFD4E0DEBF89
:1000C000CDBF11E0A0E0B1E0EAE7FCE002C005909E
:1000D0000D92A231B107D9F712E0A2E1B1E001C05F
:1000E0001D92A23FB107E1F710E0C6EBD0E004C0DB
:1000F0002297FE010E943706C43BD107C9F70E9430
:100100008D020C943B060C94000040E051EE60E040
:1001100070E08CE592E00E94A50264E670E080E069
:1001200090E00E94480461E0809100010E94BA04BE
:100130000895BF92CF92DF92EF92FF920F931F9399
:10014000DF93CF93CDB7DEB72A970FB6F894DEBF13
:100150000FBECDBF6B01DE011196E2E0F1E02AE0B7
:1001600001900D922150E1F79C0189589F4FFC01AD
:10017000849125573F4FF901B490E82FF0E0EE0F3E
:10018000FF1FEC0FFD1F0181128190E2E92EF12C7F
:10019000E00EF11EF80180A18B2980A38AE090E097
:1001A0000E947204F894F80180A19B2D90958923F8
:1001B00080A300000000000000000000000000001C
:1001C000000000000000000000000000000000002F
:1001D000000000000000000000000000000000001F
:1001E000000000000000000000000000000000000F
:1001F00000000000000000000000000000000000FF
:1002000000000000000000000000000000000000EE
:10021000000020E030E0C0FE04C0F70180818B299F
:1002200003C0F70180818923808300000000000063
:1002300000000000000000000000000000000000BE
:1002400000000000000000000000000000000000AE
:10025000000000000000000000000000000000009E
:10026000000000000000000000000000000000008E
:10027000000000000000000000000000000000007E
:10028000000000000000000000002F5F3F4F2830FA
:10029000310519F0D594C794BECFF80180A18B2900
:1002A00080A378942A960FB6F894DEBF0FBECDBF18
:1002B000CF91DF911F910F91FF90EF90DF90CF9042
:1002C000BF900895CF93DF9360E0809100010E947A
:1002D000D8046AE070E080E090E00E944804109248
:1002E0001C02C0E0D0E08091000190910101C03477
:1002F000D10531F0FE01E45EFD4F608170E002C087
:1003000060E070E00E9499002196C134D10559F750
:10031000DF91CF9108950F931F938CE592E00E9497
:10032000A202882309F4ADC08CE592E00E949F02EE
:100330009093130180931201893D910509F0A1C0AA
:100340008CE592E00E94A2028823D1F38CE592E032
:100350000E949F02809317011092150110921401C0
:100360001BC08CE592E00E94A2028823A9F00091B4
:100370001401109115018CE592E00E949F02085E25
:100380001E4FF80180838091140190911501019610
:10039000909315018093140180911401909115019F
:1003A0000497FCF2209118013091190150911A0123
:1003B000832F820F850F8093160190911B0140912E
:1003C00017019817F1F4442339F420931C0130935A
:1003D0001D0150931E0155C0842F90E0FC01EE0FCB
:1003E000FF1FE80FF91FE45EFE4F21833283019661
:1003F000FC01EE0FFF1FE80FF91FE45EFE4F508374
:1004000040C050E060E070E020E030E08CE592E039
:100410000E9469034091180150E060E070E020E024
:1004200030E08CE592E00E9469034091190150E0B0
:1004300060E070E020E030E08CE592E00E9469032B
:1004400040911A0150E060E070E020E030E08CE57F
:1004500092E00E94690340911B0150E060E070E06F
:1004600020E030E08CE592E00E94690340911601A3
:1004700050E060E070E020E030E08CE592E00E9427
:100480006903809117018823D9F410921501109205
:100490001401ACE1B1E080E090E00AC02C91E82FBB
:1004A000803420F4F0E0E45EFD4F20830196119645
:1004B000833091059CF3909315018093140128C01B
:1004C00090E09C01220F331F280F391F2F5F3F4FF1
:1004D00030931501209314010196AC01440F551F70
:1004E000480F591FD901A45EBE4F0BC08C91E22F5B
:1004F000203420F4F0E0E45EFD4F80832F5F3F4F17
:1005000011964217530794F7309315012093140165
:100510000E9462011F910F9108950E9480040E9421
:1005200085000E948B01FDCF80E191E090935D02F8
:1005300080935C020895862F0E945C0508950E94B6
:10054000750508950E9464050895CB01BA010E94C3
:10055000230508952F923F924F925F926F927F9260
:100560008F929F92AF92BF92CF92DF92EF92FF92C3
:100570000F931F93DF93CF93CDB7DEB7A0970FB63E
:10058000F894DEBF0FBECDBF1C016A017B0141158F
:1005900051056105710549F4DC01ED91FC91019073
:1005A000F081E02D60E3099554C08824992454011A
:1005B000422E55246624772401E010E00C0F1D1F05
:1005C000080D191DC701B601A30192010E94E4059F
:1005D000F80160830894811C911CA11CB11CC70107
:1005E000B601A30192010E94E405C901DA016C0180
:1005F0007D01C114D104E104F104F1F681E0E82E9B
:10060000F12CEC0EFD1EE80CF91C3E010894611C57
:10061000711CD501C4010197A109B1096C01C81869
:10062000D90814C0F601EE0DFF1D60816A3010F488
:10063000605D01C0695CD101ED91FC910190F08198
:10064000E02DC10109950894E108F1086E147F04BA
:1006500049F7A0960FB6F894DEBF0FBECDBFCF917D
:10066000DF911F910F91FF90EF90DF90CF90BF909F
:10067000AF909F908F907F906F905F904F903F9042
:100680002F900895EF92FF920F931F93CF93DF93D4
:10069000EC017A018B0177FF0FC0E881F9810190AD
:1006A000F081E02D6DE2099510950095F094E094AD
:1006B000E11CF11C011D111D2AE0B801A701CE01AA
:1006C0000E94AA02DF91CF911F910F91FF90EF90AE
:1006D0000895DC012115310541F4ED91FC91019063
:1006E000F081E02D642F099508952A30310519F421
:1006F0000E94420308950E94AA0208951F920F9239
:100700000FB60F9211242F933F934F935F936F93E4
:100710007F938F939F93AF93BF93EF93FF938091BA
:100720005E0290915F02892B29F0E0915E02F091C8
:100730005F020995FF91EF91BF91AF919F918F91CA
:100740007F916F915F914F913F912F910F900FBECD
:100750000F901F9018951F920F920FB60F921124B1
:100760002F933F934F935F936F937F938F939F93B9
:10077000AF93BF93EF93FF938091600290916102DA
:10078000892B29F0E0916002F09161020995FF91B7
:10079000EF91BF91AF919F918F917F916F915F91F9
:1007A0004F913F912F910F900FBE0F901F90189572
:1007B0001F920F920FB60F9211242F938F939F9336
:1007C000AF93BF938091620290916302A091640203
:1007D000B09165020196A11DB11D809362029093B4
:1007E0006302A0936402B0936502809166029091C7
:1007F0006702A0916802B09169028050904CAF4F9F
:10080000BF4F8093660290936702A0936802B093F3
:10081000690227C08091660290916702A0916802E8
:10082000B091690280589E43A040B0408093660218
:1008300090936702A0936802B093690280916A0264
:1008400090916B02A0916C02B0916D020196A11D76
:10085000B11D80936A0290936B02A0936C02B093D7
:100860006D028091660290916702A0916802B0913A
:10087000690281589E43A040B04060F6BF91AF919D
:100880009F918F912F910F900FBE0F901F901895F1
:10089000EF92FF920F931F937B018C018FB7F89417
:1008A00040916A0250916B0260916C0270916D02EE
:1008B0008FBF2FB7F89480916A0290916B02A0913C
:1008C0006C02B0916D022FBF841B950BA60BB70B6A
:1008D000E816F9060A071B0760F71F910F91FF90B2
:1008E000EF900895019759F0FC01EE0FFF1FEE0FF6
:1008F000FF1F32978FB7F8943197F1F78FBF0895A4
:10090000789484B5826084BD84B5816084BD85B5EA
:10091000826085BD85B5816085BDEEE6F0E08081B1
:1009200081608083E1E8F0E0808182608083808163
:1009300081608083E0E8F0E0808181608083E1EB8A
:10094000F0E0808184608083E0EBF0E08081816072
:100950008083EAE7F0E08081846080838081826028
:100960008083808181608083808180688083109211
:10097000C1000895282F30E0C90185579F4FFC0121
:10098000949129583F4FF9018491882381F0E82FF1
:10099000F0E0E859FF4FE491F0E0662329F480810C
:1009A00090958923808308958081892B8083089581
:1009B000482F50E0CA0181569F4FFC012491CA0183
:1009C00085579F4FFC01949149585F4FFA0134912C
:1009D0003323C1F1222331F1233021F480918000AF
:1009E0008F7705C0243031F4809180008F7D809313
:1009F000800018C0213019F484B58F7704C02230EC
:100A000021F484B58F7D84BD0DC0263021F4809102
:100A1000B0008F7705C0273029F48091B0008F7D1A
:100A20008093B000E32FF0E0E359FF4FE491F0E052
:100A3000662329F48081909589238083089580819D
:100A4000892B80830895EF92FF920F931F937B0170
:100A50008C0122E030E040E050E00E940606205C7D
:100A60003D4B404F5F4FCA01B901A80197010E9459
:100A70000606C901DA010197A109B109292F3A2F08
:100A80004B2F552747FD5A950196A11DB11D209367
:100A9000C50081508093C400E1ECF0E0808180616A
:100AA00080838081886080838081806880831F91BB
:100AB0000F91FF90EF900895982F8091C00085FFCF
:100AC000FCCF9093C600089580916E0290916F02C2
:100AD00080589F4F2091700230917102821B930BBE
:100AE00060E870E00E94D105089540917002509135
:100AF000710280916E0290916F028417950719F42C
:100B00002FEF3FEF0FC0FA01EE58FD4F2081CA01D1
:100B1000019660E870E00E94D10590937102809385
:100B2000700230E0C90108951F920F920FB60F9224
:100B300011242F933F934F935F936F937F938F93E2
:100B40009F93AF93BF93EF93FF934091C600E091C3
:100B50006E02F0916F02CF01019660E870E00E9492
:100B6000D1059C018091700290917102281739077C
:100B700039F0EE58FD4F408330936F0220936E02A0
:100B8000FF91EF91BF91AF919F918F917F916F9165
:100B90005F914F913F912F910F900FBE0F901F903B
:100BA000189597FB092E07260AD077FD04D049D067
:100BB00006D000201AF4709561957F4F0895F6F7DE
:100BC000909581959F4F0895A1E21A2EAA1BBB1BF9
:100BD000FD010DC0AA1FBB1FEE1FFF1FA217B30709
:100BE000E407F50720F0A21BB30BE40BF50B661F1F
:100BF000771F881F991F1A9469F7609570958095E3
:100C000090959B01AC01BD01CF01089597FB092E82
:100C100005260ED057FD04D0D7DF0AD0001C38F4CB
:100C200050954095309521953F4F4F4F5F4F089518
:100C3000F6F790958095709561957F4F8F4F9F4FF8
:100C40000895AA1BBB1B51E107C0AA1FBB1FA61713
:100C5000B70710F0A61BB70B881F991F5A95A9F765
:100C600080959095BC01CD010895EE0FFF1F059072
:0A0C7000F491E02D0994F894FFCFF1
:100C7A00050000000000050008000B00000000004D
:020C8A009B02CB
:00000001FF
